:020000040800F2
:1000000000C000205D1C0008E51B0008E71B00087D
:10001000E91B0008EB1B0008ED1B000800000000B6
:10002000000000000000000000000000EF1B0008BE
:10003000F11B000800000000F31B0008F51B00087E
:10004000A51C0008A51C0008A51C0008A51C00088C
:10005000A51C0008A51C0008A51C0008A51C00087C
:10006000A51C0008A51C0008A51C0008A51C00086C
:10007000A51C0008A51C0008A51C0008A51C00085C
:10008000A51C0008A51C0008A51C0008A51C00084C
:10009000A51C0008A51C0008A51C0008A51C00083C
:1000A000A51C0008A51C0008A51C0008A51C00082C
:1000B000A51C0008A51C0008A51C0008A51C00081C
:1000C000A51C0008A51C0008A51C0008A51C00080C
:1000D000A51C0008F91B0008A51C0008A51C0008A9
:1000E000A51C0008A51C0008A51C0008A51C0008EC
:1000F000A51C0008A51C0008A51C0008A51C0008DC
:10010000A51C0008A51C0008A51C0008A51C0008CB
:10011000A51C0008A51C0008051C0008A51C00085B
:10012000A51C0008A51C0008A51C0008A51C0008AB
:1001300000000000000000000000000000000000BF
:1001400000000000000000000000000000000000AF
:10015000000000000000000000000000000000009F
:10016000000000000000000000000000000000008F
:10017000000000000000000000000000000000007F
:10018000000000000000000000000000000000006F
:10019000000000000000000000000000000000005F
:1001A000000000000000000000000000000000004F
:1001B000000000000000000000000000000000003F
:1001C000000000000000000000000000000000002F
:1001D000000000000000000000000000000000001F
:0401E0005FF8E0F1F3
:1001E40010B5054C237833B9044B13B10448AFF36D
:1001F40000800123237010BD78000020000000005F
:10020400B82D000808B5034B1BB103490348AFF3ED
:10021400008008BD000000007C000020B82D00080C
:10022400D0400B1CD1409C46203AD3401843524244
:10023400634693401843704738B50E4B054618780B
:100244004FF47A73B3FBF0F30B4A1068B0FBF3F08E
:1002540000F09EF8044658B90F2D09D802462946E5
:100264004FF0FF3000F054F8044B20461D6038BDB9
:10027400012038BD000000200C00002004000020F4
:10028400074A08B51368032043F01003136000F015
:100294002DF80020FFF7D0FF01F030FC002008BD4E
:1002A40000200240034A044B11681B780B4413607E
:1002B400704700BFD000002000000020014B1868E8
:1002C400704700BFD000002038B50446FFF7F6FFA2
:1002D4000546631C1EBF044B1B78E418FFF7EEFFB2
:1002E400401B8442FAD838BD00000020074A0002AF
:1002F400D36800F4E06023F4E0631B041B0C43F0B8
:10030400BF6343F400330343D360704700ED00E060
:10031400174B30B5DC68C4F30224C4F10703251D70
:10032400042B28BF0423062D4FF0010598BF002499
:1003340005FA03F303F1FF3388BF033C1940A140DE
:1003440005FA04F4013C2240002842EA01024FEA83
:100354000212AFBF00F16040064B00F00F00D2B2B2
:10036400A5BFD2B200F561401A5480F8002330BD15
:1003740000ED00E014ED00E00123420900F01F004D
:1003840003FA00F0014B43F82200704700E100E05B
:100394000138B0F1807F0AD2F021064B064A58603A
:1003A40082F823100020072298601A607047012009
:1003B400704700BF10E000E000ED00E090F821304D
:1003C40010B5022B03D004238363012010BD0368FE
:1003D4001A6822F00E021A601A6822F001021A60EA
:1003E400294A934224D902F56272934219D01432F5
:1003F400934218D01432934217D0143293420CBF54
:100404004FF480534FF48033204A53600123002477
:1004140080F82130436B80F820409BB398472046F6
:1004240010BD0123F0E71023EEE74FF48073EBE7F0
:1004340017498B4216D014318B4215D014318B429C
:1004440014D014318B4214D014318B4214D0143193
:100454008B4214D0934214BF4FF480334FF0807317
:100464000C4AD2E70123FBE71023F9E74FF480732A
:10047400F6E74FF48053F3E74FF48033F0E74FF49B
:100484008013EDE7184610BD8000024000040240CE
:100494000800024000000240114AD36813F0100320
:1004A40005D01049CB6943F00203CB611023D26815
:1004B400500706D50B4943F00403CA6942F0010210
:1004C400CA61074AD169C90708D50648C16941F01C
:1004D4000401C161D16921F00101D161D360704788
:1004E40000200240D8000020064B186910F080005C
:1004F40007D0054A5A6002F188325A601869C0F37D
:10050400C01070470020024023016745034A0020C1
:10051400136943F080031361704700BF0020024059
:10052400F8B50646FFF7CAFE114C07462546E368B0
:10053400D80712D4E368990644BF2023E360EB682C
:10054400DA0606D4EB69DB0703D4E86810F004008C
:1005540002D0FFF7A1FF0120F8BD731CE7D00EB94C
:100564000320F8BDFFF7AAFEC01B8642DFD2F7E7DF
:10057400002002402DE9F84F1F4C9946237E054682
:10058400012B0F46904633D001234CF25030237692
:10059400FFF7C6FF40BB012D03D0022D0CBF02257F
:1005A40004250026B246DFF854B0320140464946DD
:1005B400FFF736FEC4F81CA0DBF8103080B243F01D
:1005C4000103CBF8103027F816004CF25030FFF737
:1005D400A7FFDBF8103023F00103CBF8103018B973
:1005E4000136F3B29D42E0D800232376BDE8F88FAC
:1005F4000220BDE8F88F00BFD80000200020024090
:100604000022064BDA61064B1A6942F004021A61B1
:100614001A6942F040021A61704700BFD8000020F6
:10062400002002400022064BDA61064B1A6942F0B0
:1006340002021A6158611A6942F040021A61704755
:10064400D8000020002002402DE9F041234D074648
:100654002B7E8846012B3DD0012403682C76022B87
:100664004CF2503013D1FFF75BFF20B1012000237F
:100674002B76BDE8F081FFF7C3FF4CF25030FFF753
:100684004FFF174A136923F004031361EFE7FFF7E1
:1006940047FF0028EAD14FF0FF33C8F80030204666
:1006A400BE680F4CFA68BB6803EBC2239E42DED2DD
:1006B4003046FFF7B7FF4CF25030FFF731FF2369A4
:1006C40023F00203236110B1C8F80060CFE706F5F8
:1006D4000066E7E70220BDE8F08100BFD8000020F3
:1006E400002002402DE9F74F002216466C4F6D4B57
:1006F400DFF8B8E1DFF8B8C14FF001080C6808FA78
:1007040006F808EA0404A04540F085804D68122DDF
:1007140000F0B78000F28D80022D00F0AF8000F26F
:100724008180002D00F09180012D00F0A5804FF014
:100734000F09FF2C93BF824606F18045083DD0F88F
:1007440000B092BFB500D0F804B0AD0009FA05F8C6
:100754002BEA080802FA05F588BF00F1040A48EA02
:100764000505CAF80050D1F804A01AF0805F52D0F1
:10077400BD6926F0030845F00105BD61BD6908F1B6
:10078400804805F00105019508F5803806F0030B53
:10079400019D4FEA8B0BD8F8085009FA0BF925EAAA
:1007A4000909414DA84271D005F58065A8426FD072
:1007B40005F58065A8426DD005F58065A8426BD02B
:1007C40005F58065A84269D070450CBF052506254E
:1007D40005FA0BF545EA0905C8F808501D681AF42E
:1007E400803F14BF2543A5431D605D681AF4003F94
:1007F40014BF2543A5435D609D681AF4801F14BF90
:100804002543A5439D60DD681AF4001F14BF2C43E3
:1008140025EA0404DC600136102E7FF46DAF03B0CA
:10082400BDE8F08F032D25D0112D80D1CA68043284
:100834007DE7654509D012D8DFF878904D4504D09E
:1008440009F580394D457FF472AF8A68E2B1012A17
:100854000CBFC0F81080C0F81480082267E7DFF8E6
:1008640058904D45F1D009F580394D45EDD0A9F5A5
:100874008019E7E700225AE7CA6858E7CA680832CD
:1008840055E7CA680C3252E7042250E700259FE777
:1008940001259DE702259BE7032599E7042597E7B2
:1008A400001002400004014000080140001C014007
:1008B4000000211000001110000031100AB1016184
:1008C40070470904FBE7C3685940C16070470000E2
:1008D40003682DE9F341DB07054610D42B689F0715
:1008E4005ED42B68190700F195802B685A0700F134
:1008F400BF80EA69002A40F02D81002014E0904C6A
:10090400636803F00C03042B07D0636803F00C0343
:10091400082B0CD16368DE0309D523689C03DDD55D
:100924006B68002BDAD1012002B0BDE8F0816B685E
:10093400B3F5803F10D1236843F480332360FFF77D
:10094400BDFC064623689803C8D4FFF7B7FC801B98
:100954006428F7D90320E7E79BB9236823F480339D
:100964002360236823F480232360FFF7A7FC064653
:1009740023689903B2D5FFF7A1FC801B6428F7D93B
:10098400E8E7B3F5A02F236803D143F48023236061
:10099400D1E723F480332360236823F48023CDE755
:1009A400674C636813F00C0F07D0636803F00C0303
:1009B400082B10D16368DA030DD423689B0702D592
:1009C4002B69012BAFD123686A6923F0F80343EA4A
:1009D400C203236085E72A695A4B6AB101221A606F
:1009E400FFF76CFC064623689F07ECD4FFF766FC10
:1009F400801B0228F7D9ADE71A60FFF75FFC0646B3
:100A0400236898077FF56DAFFFF758FC801B022819
:100A1400F6D99FE7AA694A4C4B4BDAB101221A6016
:100A2400FFF74CFC0646636A9B070DD54FF4FA5258
:100A3400464B1B68B3FBF2F3019300BF019B5A1EA4
:100A44000192002BF9D150E7FFF738FC801B0228F4
:100A5400E9D97FE71A60FFF731FC0646636A9F070E
:100A64007FF543AFFFF72AFC801B0228F6D971E714
:100A7400334CE369D80024D40127E36943F080535D
:100A8400E361E36903F080530093009B304E3368C5
:100A9400D90518D5EB68012B26D1236A43F001034D
:100AA4002362FFF70BFC41F288368046236A9B07DA
:100AB4003FD5002F3FF41DAFE36923F08053E3617A
:100AC40017E70027E2E7336843F480733360FFF7E6
:100AD400F5FB80463368DA05DCD4FFF7EFFBA0EBC7
:100AE40008006428F6D935E7ABB9236A41F288389F
:100AF40023F001032362236A23F004032362FFF734
:100B0400DDFB0646236A9807D3D5FFF7D7FB801B86
:100B14004045F7D91EE7052B236A03D143F00403AC
:100B24002362BAE723F001032362236A23F0040358
:100B3400B6E7FFF7C3FBA0EB0800B042B6D909E75C
:100B44000010024000004242800442420C00002097
:100B540000700040224C636803F00C03082B3FF440
:100B6400E2AE00231F4E022A33602BD1FFF7A6FB0F
:100B74000746236899011FD42B6AB3F5803F05D13A
:100B84006268A96822F400320A436260696A626892
:100B94000B4322F474121343636001233360FFF7A1
:100BA4008DFB054623689A013FF5A7AEFFF786FB48
:100BB400401B0228F6D9CDE6FFF780FBC01B0228B4
:100BC400D7D9C7E6FFF77AFB054623689B017FF573
:100BD40094AEFFF773FB401B0228F6D9BAE600BFB8
:100BE400001002406000424230B5194B87B002AC9D
:100BF40003F11005224618685968083303C2AB4252
:100C04001446F7D101238DF80430022311498DF8DD
:100C140005304B6803F00C02082A17D1C3F3834252
:100C240006A80244DB0312F8102C0CD54B680A48C2
:100C3400C3F34043504306AA134413F8143CB0FBD7
:100C4400F3F007B030BD05485043FAE70248F8E72F
:100C5400D02D00080010024000127A0000093D0067
:100C6400544A2DE9F0411368054603F007038B420B
:100C74000E462AD329688C0734D4CA0747D44D4A70
:100C8400136803F007039E42C0F082802A684A4C2E
:100C940012F0040F40F08780130706D563682A69B1
:100CA40023F4605343EAC2036360FFF79DFF636864
:100CB400424AC3F30313D35CD840414B186000206D
:100CC400FFF7BAFA0020BDE8F081136823F00703A8
:100CD4000B431360136803F007039942CAD0012041
:100CE400BDE8F081344B11F0040F1EBF5A6842F482
:100CF400E0625A60080742BF5A6842F460525A6080
:100D04005A68A86822F0F00202435A60B5E76A689C
:100D1400294C012A23681CD113F4003FDFD06368F7
:100D240041F2883823F0030313436360FFF7C6FAE4
:100D34006B680746012B14D1636803F00C03042B82
:100D44009DD0FFF7BBFAC01B4045F5D90320BDE891
:100D5400F081022A02D113F0007FDFE713F0020FC3
:100D6400DCE7022B0FD1636803F00C03082B86D059
:100D7400FFF7A4FAC01B4045F5D9E7E7FFF79EFA51
:100D8400C01B4045E2D8636813F00C0FF6D176E738
:100D9400136823F0070333431360136803F0070356
:100DA4009E429CD172E76368E96823F4E0630B43D5
:100DB400636071E70020024000100240CE2E00085C
:100DC4000C000020044B054A5B68C3F30223D35C88
:100DD400034A1068D840704700100240DE2E000815
:100DE4000C000020044B054A5B68C3F3C223D35CA8
:100DF400034A1068D840704700100240DE2E0008F5
:100E04000C00002003680020DA6842F00102DA6076
:100E14001A6842F001021A607047704770477047C1
:100E24007047036810B51A69044691070ED5DA684D
:100E340092070BD56FF002021A6101229B690277B7
:100E44009B0777D0FFF7EAFF0023237723681A690B
:100E5400500710D5DA6851070DD56FF004021A61F6
:100E640002229B69227713F4407F204668D0FFF763
:100E7400D5FF0023237723681A6912070FD5DA6890
:100E840010070CD56FF008021A610422DB6922777F
:100E9400990720465AD0FFF7C1FF00232377236820
:100EA4001A69D20610D5DA68D0060DD56FF0100293
:100EB4001A610822DB69227713F4407F20464BD065
:100EC400FFF7ACFF0023237723681A69D10708D5FD
:100ED400DA68D20705D56FF0010220461A6100F0E6
:100EE40067FB23681A69100608D5DA68110605D568
:100EF4006FF0800220461A6100F0BFF823681A6977
:100F0400520608D5DA68500605D56FF0400220462F
:100F14001A61FFF785FF23681A69910622D5DA68FA
:100F240092061FD56FF020022046BDE810401A61DA
:100F340000F0A2B8FFF771FF2046FFF770FF83E7C8
:100F4400FFF76BFF2046FFF76AFF92E7FFF765FFA5
:100F54002046FFF764FFA0E7FFF75FFF2046FFF797
:100F64005EFFAFE710BD0000244A0368904212D030
:100F740002F5006290420ED0B0F1804F0BD0A2F582
:100F84009832904207D002F58062904203D002F575
:100F9400806290421DD14A6823F070031343174ABC
:100FA400904212D002F5006290420ED0B0F1804F10
:100FB4000BD0A2F59832904207D002F5806290429D
:100FC40003D002F58062904203D1CA6823F44073CF
:100FD40013434A6923F08003134303608B68C3629D
:100FE4000B688362054B984203D003F50063984273
:100FF40001D10B690363012343617047002C014055
:1010040010B50446A0B190F83D3003F0FF021BB9BF
:1010140080F83C2000F094FD0223206884F83D30E1
:10102400211DFFF7A1FF0123002084F83D3010BDEE
:10103400012010BD90F83C3010B5012B4FF0020395
:1010440018D080F83D3003680C685A68496822F06B
:1010540070025A605A6822435A609A6822F08002E9
:101064009A609A680A439A60012380F83D3000230D
:1010740080F83C30184610BD704770470368DA6842
:1010840022F49072DA605A6922F001025A61202334
:1010940080F83A30704700002DE9F0470568C268CF
:1010A4002B69016923F4405313432B618368EA6875
:1010B4000B43416922F4B05222F00C020B43134358
:1010C400EB606B69826923F4407313436B61404B9B
:1010D40081469D424FF0190446D1FFF783FE04FB7D
:1010E40000F3D9F804604FF06408B600B3FBF6F3DC
:1010F400B3FBF8F31E01FFF775FE6043D9F8043023
:101104009B00B0FBF3F7FFF76DFE6043D9F80430A2
:101114009B00B0FBF3F3B3FBF8F308FB13731B0161
:101124003233B3FBF8F303F0F007FFF75BFE6043E1
:10113400D9F804209200B0FBF2FAFFF753FE6043A3
:10114400D9F804309B00B0FBF3F3B3FBF8F308FBCE
:1011540013A31B013233B3FBF8F303F00F033B4338
:101164003344AB60BDE8F087FFF72CFE04FB00F3CB
:10117400D9F804604FF06408B600B3FBF6F3B3FB90
:10118400F8F31E01FFF71EFE6043D9F804309B00FC
:10119400B0FBF3F7FFF716FE6043D9F804309B0069
:1011A400B0FBF3F3B3FBF8F308FB13731B01323307
:1011B400B3FBF8F303F0F007FFF704FE6043D9F83C
:1011C40004209200B0FBF2FAFFF7FCFDB7E700BF82
:1011D40000380140F8B504460E4617461D462168FE
:1011E4000B6836EA030301D10020F8BD6B1CF7D06D
:1011F40095B923680320DA6822F4D072DA605A6958
:1012040022F001025A61202384F8393084F83A30FC
:10121400002384F83830F8BDFFF750F8C01B85422E
:10122400DDD2E6E710B5044640B390F8393003F058
:10123400FF021BB980F8382000F096FC24232268B2
:1012440084F83930D368204623F40053D360FFF781
:1012540023FF236800201A6922F490421A615A6914
:1012640022F02A025A61DA6842F40052DA6020233A
:10127400E06384F8393084F83A3010BD012010BDA1
:101284002DE9F0411F4690F839300446202B0D46D5
:1012940090464ED1002949D0002A47D090F83830E2
:1012A400012B46D0012380F838300023C363212367
:1012B40080F83930FFF702F80646A4F82480A4F831
:1012C4002680E38C9BB26BB93B46324640212046D4
:1012D400FFF780FFA8B9202384F8380084F8393058
:1012E400BDE8F081E38C3246013B9BB2E384A36802
:1012F4008021B3F5805F20463B460ED1FFF76AFF9D
:1013040010B10320BDE8F0812B882268C3F30803E1
:101314005360236943B90235D3E7FFF75BFF002825
:10132400EFD123682A785A600135CAE70120BDE865
:10133400F0810220BDE8F08190F83A30202B20D1D2
:10134400E9B1E2B190F83830012B1AD0C285828518
:1013540000232222C36380F83A2002688162D168A4
:1013640080F8383041F48071D1605169184641F0F9
:1013740001015161D16841F02001D1607047012021
:10138400704702207047704790F83A3010B5222B0E
:1013940036D183680169B3F5805F0268836A23D11B
:1013A4005268E9B9C2F3080223F8022B8362C48DA0
:1013B400013CA4B2C4858CB90368DA6822F0200227
:1013C400DA60DA6822F48072DA605A6922F0010283
:1013D4005A61202380F83A3000F0CAF8002010BD8A
:1013E400D2B223F8012BE1E721B9591C526881627A
:1013F4001A70DCE75268591C816202F07F02F7E739
:10140400022010BD70470000036870B51A680446D6
:101414001607D9685D6907D196065AD58D0658D541
:10142400BDE87040FFF7B0BF15F0010502D111F41B
:10143400907F4ED0D30705D5CE0542BFE36B43F072
:101444000103E363500704D51DB1E36B43F00203CA
:10145400E363930704D51DB1E36B43F00403E36333
:10146400160704D51DB1E36B43F00803E363E36B94
:10147400002B66D0950604D5880602D52046FFF7D2
:1014840083FF236820465D69E26B110702D415F0DF
:1014940040051AD0FFF7F2FD23685A69520610D5A9
:1014A4005A69606B22F040025A6150B1254B436384
:1014B400FEF784FF002844D0606BBDE87040436BA6
:1014C40018472046FFF79EFF70BDFFF79BFFE563BB
:1014D40070BD160627D50D0625D594F83920212A86
:1014E4002FD1A268B2F5805F226A17D11188C1F3A7
:1014F40008015960216979B902322262E28C013A09
:1015040092B2E284EAB9DA6822F08002DA60DA6838
:1015140042F04002DA6070BD0132EEE7511C2162F4
:1015240012785A60EAE750060BD54A0609D5DA68FC
:10153400204622F04002DA60202384F83930FFF795
:1015440022FF70BD4D15000808B50023406AC3850D
:10155400C384FFF757FF08BD08B5FEF7C5FF342263
:10156400024BDA60BDE80840FEF7D0BF002002401D
:1015740002680A4B9A420FD1094A0A49136808784B
:101584000949C8540133632B88BF002305491360FC
:1015940006480122FFF7D0BE704700BF0038014063
:1015A400B8000020C000002088010020FC000020BA
:1015B4000268084B9A420BD1074A1368013313603F
:1015C400064A136801331360054A13680133136034
:1015D400704700BF00100040B0000020A8000020A9
:1015E400A40000200A460A2301460148FFF748BE2A
:1015F400FC00002010B514460A230248FFF740FE01
:10160400204610BDFC0000202DE9F04100240746CF
:101614002646104DDFF84080BB78023B9C4202DB3B
:101624003046BDE8F0813B19DA781B79296802EB72
:10163400032292B200230120FEF79CFF18B140461A
:1016440000F0D0FB01262B68023402332B60E4B295
:10165400E2E700BF08000020202E0008002373B535
:10166400164D174C2B60174B0646AB601F23EB60DF
:10167400E36923F01003E361FEF736FF124B1A7897
:101684004AB90122114928461A70FEF7DDFF10B14C
:101694000F4800F0A7FB3046FFF7B6FF0546FEF7FC
:1016A40035FF2846E36943F01003E361E36903F07F
:1016B40010030193019B02B070BD00BF9400002091
:1016C4000010024000400008B4000020AC000020DC
:1016D4002C2E000870B5064C064E074D2278214684
:1016E4003046013400F00AFBAC42F7D170BD00BFB4
:1016F40000400008122E000810400008B0B50D4A42
:1017040000AFD3690C4823F01003D36100F06AFBE7
:101714000A4B0B4A1B680B4C0B481360236000F008
:1017240061FB0A4B1B6883F308882368BD46BDE848
:10173400B0401847001002403B2E00080440000847
:101744003C010020840100204D2E000800400008C8
:1017540073B50446254BA17818681B7900908DF861
:10176400043063185A78601C00F0ABF901280BD0E0
:1017740000231F4EA2785D1C0232DBB29A422FDA9C
:101784001C4800F02FFB0CE011238DF80130637826
:10179400DD2B01D0EE2B07D12046FFF75FFF012898
:1017A40002D122238DF801309DF802100DF10100C1
:1017B40000F06CF963788DF80300EE2B08D00A2B47
:1017C40006D09DF8021068460331C9B2FFF70AFF3C
:1017D4006378EE2B02D1084800F004FB02B070BD20
:1017E400E15C304600F08AFA2B46C3E7E02D00089E
:1017F400EA2D0008F02D0008012E000810B590B065
:101804002822002106A800F071FA0021142201A860
:1018140000F06CFA022401224FF4803306A80692E9
:1018240007930A920E930D94FFF752F80F230021A9
:1018340001934FF4806301A80294039104930591EA
:10184400FFF70EFA10B010BD2DE9F047CAB00AAF89
:10185400FF220021384600F049FA774B002418682B
:101864001B7904908DF81430FEF70AFDFFF7C6FFCC
:101874001022002106A800F039FA704B4FF4004101
:101884009A696F4842F010029A619A694FF0010810
:1018940002F010020192019A9A696A4E42F0200203
:1018A4009A619A69684D02F020020292029A9A693A
:1018B40042F004029A619B69002203F0040303933B
:1018C400039BFEF7FBFF4FF400430693022306A994
:1018D4005B48CDF81C8009930894FEF703FF40F29F
:1018E4003F635A4A304686E80C000923B460F3602B
:1018F400B46106940794FFF783FB06A93046069467
:101904000794FFF797FB4FF4E1335149284685E8E4
:101914000A000C23AC606B61EC602C61AC61EC617F
:10192400FFF780FC224621463620FEF7F1FC3620E4
:10193400FEF722FD224621462520FEF7E9FC25205C
:10194400FEF71AFD3046FFF75DFA42464149284644
:10195400FFF7F2FC404B21461B68404E986800F0AC
:1019640049FA3F4800F03EFA3E4800F03BFA3E4A4E
:101974003E493F4800F0C2F93E4800F033FA384887
:1019840000F030FAFFF7E8FDFFF7A4FE9DF812100F
:101994000DF1110000F07AF88DF813006420FEF7C1
:1019A40093FC9DF8121004A80331C9B2FFF71AFE84
:1019B4002546B146DFF8888040F6B83332689A424B
:1019C40001D9FFF79BFE2C4A2C4B11681B689942E6
:1019D4001ED02B4C481C615C6B1C79550021DBB27A
:1019E4001D466328106088BF1160264A1160254B8C
:1019F4001B68642B1ED900253846FFF7A9FE642214
:101A04000021384600F072F92C46C9F8005001E074
:101A1400002CECD1DFF870A0DAF80030B3F5FA7FCF
:101A2400CAD94FF400414046FEF74DFF0023CAF8DF
:101A34000030C1E70124EDE7E52D00080010024065
:101A44000010014040010020FC0000200010004074
:101A540000380140C000002010000020A400002035
:101A6400532E00087D2E00088A2E0008932E0008AD
:101A74009F2E0008B02E0008BC000020B8000020F3
:101A840088010020B0000020A800002010B5FF232A
:101A94000446221AD2B2914201D8184610BD14F855
:101AA400012B5340082213F0800F02F1FF324FEA5A
:101AB400430318BF83F0310312F0FF02DBB2F2D10B
:101AC400E7E730B5FF2305462C1AE4B2A14203D858
:101AD4009B1A5842584130BD15F8014B6340082405
:101AE40013F0800F04F1FF344FEA430318BF83F06F
:101AF400310314F0FF04DBB2F2D1E5E70E4B82B000
:101B04009A6942F001029A619A6902F00102009214
:101B1400009ADA6942F08052DA61DB69074A03F01D
:101B240080530193019B536823F0E06343F0806387
:101B3400536002B0704700BF001002400000014033
:101B44000268084B82B09A420AD103F50033DA697D
:101B540042F01002DA61DB6903F010030193019B88
:101B640002B070470010004010B5044686B0102241
:101B7400002102A800F0BAF82268174B9A4228D133
:101B840003F558439A6902A942F480429A619A691A
:101B9400124802F480420092009A9A6942F00402C8
:101BA4009A619B6903F004030193019B4FF4007352
:101BB40002930223039303230593FEF793FD4FF44B
:101BC40080630293002302A9044803930493FEF75D
:101BD40089FD06B010BD00BF003801400008014077
:101BE4007047FEE7FEE7FEE7FEE770477047704781
:101BF400FEF758BB0148FFF707BC00BFFC000020FC
:101C04000148FFF70EB900BF400100200F4B1A68CE
:101C140042F001021A6059680D4A0A405A601A6873
:101C240022F0847222F480321A601A6822F480222C
:101C34001A605A6822F4FE025A604FF41F029A6036
:101C44004FF00062034B9A60704700BF00100240DF
:101C54000000FFF800ED00E0002103E00B4B5B58AF
:101C6400435004310A480B4B42189A42F6D30A4AAD
:101C740002E0002342F8043B084B9A42F9D3FFF7F1
:101C8400C5FF00F00FF8FFF7DFFD7047882F00084D
:101C94000000002074000020780000208C02002046
:101CA400FEE7000070B500250C4E0D4CA41BA410DB
:101CB400A54209D101F07EF800250A4E0A4CA41B66
:101CC400A410A54205D170BD56F8253098470135BA
:101CD400EEE756F8253098470135F2E7802F0008E3
:101CE400802F0008802F0008842F00080346024438
:101CF400934200D1704703F8011BF9E70FB40A4B74
:101D040013B51C6824B1A36913B9204600F0DAFAAC
:101D140005AB049AA1682046019300F09BFC02B035
:101D2400BDE8104004B070471000002070B50E46A6
:101D3400054618B183690BB900F0C4FAAB69AC6805
:101D440013B9284600F0BEFA234B9C4217D16C68A5
:101D5400A3891B071DD52369DBB1013EA36816F8CF
:101D6400011F013BA360E9B9002B2EDA22460A21A8
:101D7400284600F0F5F8013011D00A2070BD174B49
:101D84009C4201D1AC68E3E7154B9C4208BFEC6868
:101D9400DEE72146284600F035F90028DDD04FF073
:101DA400FF3070BD002B04DAA269934206DB0A29D6
:101DB40004D023685A1C22601970CFE722462846B3
:101DC40000F0CEF80130C9D1E9E70A2023685A1C93
:101DD4002260187070BD00BF0C2F00082C2F000863
:101DE400EC2E0008024B01461868FFF79FBF00BFA6
:101DF4001000002000294FF480630CBF022200224F
:101E040000F000B82DE9F7431D46514B04461E6807
:101E14000F46904626B1B36913B9304600F052FA22
:101E24004C4B9C4252D17468B8F1020F06D0B8F101
:101E3400010F00F28980002DC0F2868021463046D1
:101E440000F0D6F9616B41B104F14403994202D028
:101E5400304600F02DFB002363630023A36163601D
:101E6400A3891B0603D52169304600F021FBA38911
:101E7400B8F1020F23F44A6323F00303A3815DD076
:101E840001AB6A462146304600F0A6FAA3891843FE
:101E9400A0812DBB009D284600F002FB07460028C8
:101EA4004ED1DDF80090A9453CD14FF0FF30A38915
:101EB40043F00203A3810023A36004F147032360DA
:101EC40023610123636103B0BDE8F083224B9C428C
:101ED40001D1B468A8E7214B9C4208BFF468A3E78A
:101EE400002FD8D0B36913B9304600F0EBF9B8F13C
:101EF400010F08BFA389276004BF43F00103A38136
:101F0400A389276113F0080065611BD013F0010059
:101F14004FF000031FBF6D42A360A561184608BFC0
:101F2400A560D0E7484600F0BBFA07460028BCD0BD
:101F3400A3894D4643F08003A381D3E70020B6E78D
:101F4400A946F5E7A060BEE74FF0FF30BBE700BF4E
:101F5400100000200C2F00082C2F0008EC2E000885
:101F6400F8B50E461446054618B183690BB900F05E
:101F7400A9F9214B9C422AD16C68A369A360A38967
:101F84001A072ED5236963B323692068F6B2C01AF1
:101F940063693746984204DB2146284600F028F955
:101FA40028BBA3680130013BA36023685A1C22604C
:101FB4001E706369984204D0A389DB0719D50A2EE1
:101FC40017D12146284600F013F990B10FE00B4BCE
:101FD4009C4201D1AC68D0E7094B9C4208BFEC6835
:101FE400CBE72146284600F00DF80028CCD04FF06E
:101FF400FF373846F8BD00BF0C2F00082C2F00080F
:10200400EC2E0008324B70B51D6806460C4625B10F
:10201400AB6913B9284600F055F92E4B9C420FD1F9
:102024006C68B4F90C309AB215072CD4D00611D4CC
:102034000922326043F04003A3814FF0FF3070BDAA
:10204400254B9C4201D1AC68EBE7244B9C4208BF72
:10205400EC68E6E7510712D5616B41B104F1440322
:10206400994202D0304600F023FA00236363A38927
:1020740023F02403A3810023636023692360A389DD
:1020840043F00803A38123694BB9A38903F42073A4
:10209400B3F5007F03D02146304600F0C1F9A28990
:1020A40012F001030CD00023A36063695B42A361B7
:1020B400236953B9B4F90C3013F08000BAD170BD60
:1020C400920758BF6369A360F2E70020F7E700BFF7
:1020D400100000200C2F00082C2F0008EC2E000804
:1020E4008A892DE9F041054610070C465AD44B68FD
:1020F400002B05DC0B6C002B02DC0020BDE8F0811A
:10210400E66A002EF9D0002312F480522F682B6067
:1021140033D0606DA3895A0705D56368C01A636B11
:102124000BB1236CC01A00230246E66A216A2846D2
:10213400B047431CA38906D129681D294BD82B4AD3
:10214400CA40D60747D5002262602269D9042260BA
:1021540004D5421C01D12B6803B96065616B2F6003
:102164000029CAD004F14403994202D0284600F061
:102174009FF900206063BDE8F081216A01232846AD
:10218400B047411CC6D12B68002BC3D01D2B01D0F6
:10219400162B01D12F60B0E7A38943F04003A3813C
:1021A400BDE8F0810F69002FA7D0930718BF002363
:1021B4000E6808BF4B69A6EB07080F608B60B8F187
:1021C400000F9ADD43463A46216A2846A66AB0477C
:1021D400002807DCA38943F04003A3814FF0FF30BC
:1021E400BDE8F0810744A8EB0008E8E701004020BF
:1021F40038B50B6905460C46DBB118B183690BB9D8
:1022040000F060F80C4B9C4209D16C68B4F90C30B6
:102214007BB121462846BDE83840FFF761BF074B34
:102224009C4201D1AC68F1E7054B9C4208BFEC68C5
:10223400ECE7002038BD00BF0C2F00082C2F00084D
:10224400EC2E0008014900F0A9B800BFF5210008F0
:10225400002310B5044603604360836081814366B4
:10226400C281036143618361194608225C30FFF730
:102274003DFD054B24626362044BA362044BE3629D
:10228400044B236310BD00BFD52B0008F72B0008B7
:102294002F2C0008532C000870B568254A1E55439E
:1022A4000E4605F1740100F04FF9044640B10021D7
:1022B40080E842000C30A06005F16802FFF716FDCB
:1022C400204670BD836910B5044633BB8364C36480
:1022D4000365124B124A1B688262984204BF0123B1
:1022E400836100F01FF86060204600F01BF8A060D6
:1022F400204600F017F80022E06004216068FFF730
:10230400A7FF01220921A068FFF7A2FF02221221E0
:10231400E068FFF79DFF0123A36110BDE82E0008CC
:1023240049220008F8B51C4B07461E68B36913B967
:102334003046FFF7C7FF4836B4687368013B03D5DE
:10234400336833B13668F7E7B4F90C506DB16834CB
:10235400F4E704213846FFF79FFF30600028F1D1ED
:102364000C2304463B602046F8BD4FF6FF73E3811F
:1023740001236566A3812560A560656025616561AB
:10238400A5610822294604F15C00FFF7AFFC6563F0
:10239400A563A564E564E6E7E82E00082DE9F843A3
:1023A40080468946002600F1480414B93046BDE849
:1023B400F883A5686768013F01D52468F5E7AB8910
:1023C400012B07D9B5F90E30013303D02946404615
:1023D400C84706436835EEE770B50E46B1F90E10EE
:1023E40090B0002914461D4607DA00232B60B389F8
:1023F4001A0610D44FF480630EE001AA00F04EFCDC
:102404000028F2DB029A02F47042A2F500535A4209
:102414005A412A60EEE740230020236010B070BDCB
:102424008B8973B59D0706460C4607D504F147030F
:10243400236023610123636102B070BD01AB6A466E
:10244400FFF7CAFF00990546304600F07DF848B909
:10245400B4F90C309A05EFD423F0030343F00203DC
:10246400A381E3E70D4BB362A389206043F08003AB
:10247400A381009B20616361019B5BB1B4F90E10E1
:10248400304600F01DFC28B1A38923F0030343F078
:102494000103A381A3891D43A581CDE74922000837
:1024A400024B0146186800F04FB800BF100000202E
:1024B40038B50546002943D051F8043C0C1F002BC5
:1024C400B8BFE41800F02CFC1E4A1368104633B958
:1024D400636014602846BDE8384000F022BCA34283
:1024E4000BD921686218934201BF1A685B685218BD
:1024F400226063600460EDE713465A680AB1A242A1
:10250400FAD919685818A0420BD120680144581808
:1025140082421960DED110685268014419605A6021
:10252400D8E702D90C232B60D4E7206821188A420B
:1025340001BF116852680918216062605C60C9E7D4
:1025440038BD00BFC400002070B5CD1C25F00305C4
:1025540008350C2D38BF0C25002D064601DBA94299
:1025640003D90C233360002070BD00F0D9FB234A4B
:102574001468214691B9224C23681BB9304600F0F7
:1025840017FB20602946304600F012FB431C26D17D
:102594000C233046336000F0C4FBE4E70B685B1B9C
:1025A4001AD40B2B0FD90B60CC18CD50304600F049
:1025B400B8FB04F10B00231D20F00700C31A1BD045
:1025C4005A42E25070BD8C420BBF63684B68136083
:1025D400636018BF0C46E9E70C464968CAE7C41CA7
:1025E40024F00304A04205D0211A304600F0E0FA9A
:1025F4000130CDD02560D9E770BD00BFC4000020F4
:10260400C8000020936810B4013B002B936008DAE3
:102614009469A34202DBCBB20A2B02D110BCFFF7B0
:102624009FBC1368581C10601970C8B210BC704766
:10263400F8B506460F461446D518AC4201D1002021
:1026440007E03A4614F8011B3046FFF7DBFF431C52
:10265400F3D1F8BD2DE9F04F9DB00C461746039316
:10266400064618B183690BB9FFF72CFE7C4B9C42DC
:1026740057D17468A38918075DD52369002B5AD0F4
:102684000023099320238DF8293030234FF0010BC8
:102694008DF82A30B846454615F8013B002B55D134
:1026A400B8EB070A0BD053463A4621463046FFF7AB
:1026B400BFFF013000F0C480099B5344099398F88C
:1026C4000030002B00F0BC8000234FF0FF32049355
:1026D4000793059206938DF853301A9305222978AF
:1026E400604800F00FFB05F10108049B002831D17C
:1026F400D90644BF20228DF853201A0744BF2B2249
:102704008DF853202A782A2A2CD000210A20079AEF
:10271400A84698F800300135303B092B6DD971B3C8
:1027240026E0514B9C4201D1B468A3E74F4B9C4235
:1027340008BFF4689EE721463046FFF763FC002893
:102744009ED04FF0FF301DB0BDE8F08F252BA7D0F1
:10275400A846A0E7434A4546801A0BFA00F01843FE
:102764000490BBE7039A111D12680391002A01DB50
:10277400079204E0524243F002030792049398F84C
:1027840000302E2B10D198F8013008F101012A2BCA
:1027940037D1039B08F102081A1D1B680392002B12
:1027A400B8BF4FF0FF330593314D032298F8001062
:1027B400284600F0A7FA40B14023401B03FA00F07A
:1027C400049B08F101080343049398F800100622BF
:1027D400284808F101078DF8281000F093FA002822
:1027E40034D0254B03BB039B073323F00703083383
:1027F4000393099B4B4409934CE700FB02320121EC
:1028040086E700230A2518460593884698F8002091
:102814000131303A092A03D9002BC5D00590C3E70A
:1028240005FB00200123F0E703AB00932246134B82
:1028340004A93046AFF30080B0F1FF3F8146D8D100
:10284400A3895B063FF57DAF09987CE703AB009352
:1028540022460A4B04A9304600F08AF8ECE700BF90
:102864000C2F00084C2F00082C2F0008EC2E000819
:10287400522F0008562F00080000000035260008DB
:102884002DE9F04791461F468A680B690646934234
:10289400B8BF1346C9F8003091F843200C46DDF860
:1028A400208012B10133C9F800302368990642BF71
:1028B400D9F800300233C9F80030256815F0060550
:1028C40007D104F1190AE368D9F800209B1A9D4244
:1028D4002ADB94F843302268003318BF01239206A0
:1028E4002FD404F1430239463046C047013022D088
:1028F4002368E56803F00603042B18BF0025D9F804
:1029040000204FF0000908BFAD1AA368226908BF70
:1029140025EAE5759342C4BF9B1AED181A344D4558
:102924001BD10020BDE8F0870123524639463046CA
:10293400C047013003D14FF0FF30BDE8F0870135C7
:10294400C1E73020E11881F843005A1C94F845107F
:102954002244023382F84310C3E701232246394656
:102964003046C0470130E6D009F10109D7E700003D
:102974002DE9F04317460A7E85B06E2A984606462E
:102984000C460C9B01F1430E00F0BC801AD8632A5C
:102994002ED00AD8002A00F0C880582A00F08A8075
:1029A40004F1420584F842202AE0642A01D0692A0D
:1029B400F6D121681A6811F0800F23D0111D196017
:1029C400136827E0732A00F0B48008D86F2A2AD04D
:1029D400702AE5D10A6842F020020A6003E0752AF1
:1029E40021D0782ADCD178226F4984F8452064E02C
:1029F4001A6801F14205111D1960136884F8423008
:102A04000123A3E011F0400F02F104011960D7D0B3
:102A1400B2F90030002B03DA2D225B4284F8432004
:102A240062490A2217E02068196810F0800F03D069
:102A3400081D18600B6806E010F0400F01F1040057
:102A44001860F7D00B886F2A14BF0A22082257494E
:102A5400002084F843006568002DA560C0F29C80C6
:102A6400206820F004002060002B3FD1002D40F0AE
:102A740095807546082A0BD12368DA0708D523699F
:102A840062689A42DEBF302305F8013C05F1FF3548
:102A9400AEEB05032361CDF800803B4603AA214633
:102AA4003046FFF7EDFE013055D14FF0FF3005B051
:102AB400BDE8F08381F845203C492268186812F08B
:102AC400800F00F104051D6001D0036802E0550683
:102AD400FBD50388D00744BF42F0200222601BB913
:102AE400226822F0200222601022B1E77546B3FB6F
:102AF400F2F002FB1033CB5C05F8013D03460028DD
:102B0400F5D1B7E708681A6810F0800F496904D056
:102B1400101D18601368196007E010F0400F02F1EF
:102B2400040018601368F6D01980002375462361E9
:102B3400B1E71A68111D19601568002162682846FA
:102B440000F0E0F808B1401B606063682361002373
:102B540084F843309FE723692A4639463046C04704
:102B64000130A2D023689B0707D5002504F1190979
:102B7400E368039A9B1A9D4205DBE068039B984235
:102B8400B8BF184693E701234A4639463046C04742
:102B940001308AD00135EBE7002BA7D10B7804F183
:102BA400420584F8423065E76E2F00085D2F000867
:102BB40038B50023054C05460846236000F0ECF8C0
:102BC400431C02D1236803B12B6038BD8802002066
:102BD40010B50C46B1F90E1000F0A4F80028ABBFF4
:102BE400636DA3891B1823F48053ACBF6365A38171
:102BF40010BD2DE9F0411F468B890546DB050C46C7
:102C0400164605D502230022B1F90E1000F068F82B
:102C1400A389324623F48053A381B4F90E103B46B2
:102C24002846BDE8F04100F017B810B50C46B1F9DC
:102C34000E1000F055F8431CA38915BF606523F4FA
:102C4400805343F48053A38118BFA38110BDB1F90D
:102C54000E1000F013B8000038B5054608461146BA
:102C64000022054C22601A46FEF7C4FC431C02D124
:102C7400236803B12B6038BD8802002038B50023D7
:102C8400054C05460846236000F05EF8431C02D15B
:102C9400236803B12B6038BD8802002038B50023B7
:102CA400064C054608461146236000F055F8431CBF
:102CB40002D1236803B12B6038BD00BF8802002015
:102CC40038B50023054C05460846236000F04CF84F
:102CD400431C02D1236803B12B6038BD8802002055
:102CE40038B50546084611460022054C22601A46AE
:102CF40000F042F8431C02D1236803B12B6038BDB5
:102D04008802002010B5C9B202449042034601D1A2
:102D1400002010BD1C7801308C42F6D1184610BD3D
:102D24007047704738B50546084611460022054CE1
:102D340022601A4600F028F8431C02D1236803B12C
:102D44002B6038BD880200205822024B4FF0FF3020
:102D54001A607047880200205822024B4FF0FF305F
:102D64001A607047880200205822024B00201A6023
:102D7400704700BF880200205822024B4FF0FF30FA
:102D84001A607047880200205822024B4FF0FF302F
:102D94001A60704788020020044B0246196809B97A
:102DA40003491960186802441A607047CC00002077
:102DB4008C020020F8B500BFF8BC08BC9E467047E2
:0C2DC400F8B500BFF8BC08BC9E46704784
:102DD00002030405060708090A0B0C0D0E0F10105C
:102DE000BE110200BEBE0B0200EB2530327820007F
:102DF000436865636B2053756D206572726F722036
:102E00000075706461746520436F6D706C657465E6
:102E1000200025303878203A2025303258200A000A
:102E200048414C204E4F54204F4B20004572617357
:102E300065204661696C6564200D00626F6F7420C7
:102E40006C6F61646572207374617274006A756D71
:102E50007021002A2A2A2A2A2A2A2A2A2A2A2A2ABF
:102E60002A2A2A2A2A2A2A2A2A2A2A2A2A2A2A2AC2
:102E70002A2A2A2A2A2A2A2A2A2A2A0D005247429C
:102E80002050726F6A6563740D0032303A31393AFE
:102E900030350041707220313220323031390042F9
:102EA00075696C642061742025732025730D0A00F8
:102EB000436F707972696768742028632920323003
:102EC00031392E20424C554543454C4C0D000000F5
:102ED00000000000000001020304060708090000CA
:102EE00000000102030400001400002000000000A4
:102EF00000000000000000000000000000000000D2
:102F000000000000000000000000000000000000C1
:102F100000000000000000000000000000000000B1
:102F200000000000000000000000000000000000A1
:102F30000000000000000000000000000000000091
:102F4000000000000000000000000000232D302BD6
:102F50002000686C4C00656667454647003031329A
:102F600033343536373839414243444546003031F1
:102F70003233343536373839616263646566000050
:042F8000090200083A
:042F8400E50100085B
:102F880001000000100000000040000800A24A04F0
:102F980014000020000000000C2F00082C2F00084F
:102FA800EC2E0008000000000000000000000000F7
:102FB8000000000000000000000000000000000009
:102FC80000000000000000000000000000000000F9
:102FD80000000000000000000000000000000000E9
:102FE80000000000000000000000000000000000D9
:042FF80000000000D5
:0400000508001C5D76
:00000001FF
